:020000040000FA
:10000000FF3085008316F8308500FF23900005300F
:1000100081009516151696168312073099008B15D8
:1000200020308400DF008001840ADF08031D1328CC
:100030007E20B33081000B110A30B0006720031D11
:100040002328A50A1E28F220A600250203182B2823
:100050000301A600E620260824060319312867209C
:100060002B2849208B20FF30C1003628C00F3C28A8
:10007000410885000B19F8204008370703180511BF
:10008000400835070318851040083307031805108A
:1000900036286320A700013E03195E28273084001C
:1000A000840AA20A0319A30A632080002B300406E5
:1000B000031D5028A20A0319A30A08002008A20061
:1000C0002108A300492823088A00220882008720EB
:1000D000013E031970280530A0070318A10A6728FC
:1000E000A40AA00A0319A10A8720013E03197E2849
:1000F0002008A2002108A30003010800A401013088
:10010000A100A3005A30A000A200FF380800210877
:100110008A00200882002808B1002708AF00031DCC
:1001200099282908B3002A08B5002B08B700BF0199
:1001300008000730BF000130B200B400B600330839
:1001400029020318A628B203B203003CB800350800
:100150002A020318AE28B403B403003CB9003708E0
:100160002B020318B628B603B603003CBA003808C1
:1001700039020318C22838083A023A080318C72877
:100180003808C72839083A023A08031C3908003CE5
:10019000BE00BB00BC00BD0008002408E620851E90
:1001A000CF280F30DE2005080B10630000005A3006
:1001B000DE20851ACF28851EDB28002881010B113F
:1001C0000B1DE028FF3E031DDE28080083169A0061
:1001D0009B018C131C1555309D00AA309D009C146A
:1001E0008312080083169B011C141A08831208004E
:1001F0000108B33E81000B11AE0803190529AD0BB0
:100200000529AE0B05292408E620851A0B29AC0A1E
:100210000319CD281C29FC302C0703181129AC0127
:100220001C2967204920B301B501B7018B200A3092
:10023000B000AC010830AE00BF0803194E29AF0B67
:1002400008002708AF0029083306031D29293F109D
:1002500031293808BB07031C31293E08BB07320887
:10026000B3072A083506031D3729BF103F2939086F
:10027000BC07031C3F293E08BC073408B5072B0800
:100280003706031D45293F1108003A08BD07031C26
:1002900008003E08BD073608B7070800B108031973
:1002A0005729B00B08000A30B000B10B08004920F4
:1002B0008B20080000340534FF3400340034FF3450
:1002C000003405340034FF340034FF340034053486
:1002D00000340034FF34FF3400340534003400347B
:1002E0000034FF34003405340C340C340C34FF3447
:1002F00000340534803480348034FF3400340534D5
:10030000FF34FF34FF34FF3400340534003400344C
:100310000034FF3402340134FF340034003402343A
:100320000134003400340034023401340034FF342A
:100330000034023401340034003400340234013417
:1003400000340034FF34023401340034003400340B
:10035000FF3402340034FF340034003402340034FB
:100360000034FF3400340234003400340034FF34ED
:10037000FF3400340534003400340A3400340534CA
:10038000003400340034FF34FF3472346734623494
:10039000733461345F3469346E34653474342E34AC
:1003A000613473346D342034323431342F3430348A
:1003B00033342F3432343034303437342034523400
:1003C00032342E3430342E343134283463342934EA
:1003D00020345034653474346534203447347234F6
:1003E0006934663466346934743468347334203460
:1003F00032343034303436342D34323430343034D6
:1004000037342034723467346234733461344034A6
:100410007034653474346534733477346F347234C3
:100420006C3464342E34643465346D346F346E341B
:0C0430002E3463346F342E3475346B347A
:02400E00A43FCD
:00000001FF
